:10000000500500203918000091180000D11100009F
:10001000D1110000D1110000D1110000D111000058
:10002000D1110000D1110000D11100009511000084
:10003000D1110000D111000051110000D1110000B8
:10004000F5110000F5110000F5110000F511000098
:10005000F5110000F5110000F5110000F511000088
:10006000F5110000F5110000F5110000F511000078
:10007000F5110000F5110000F5110000F511000068
:10008000F5110000F5110000F5110000F511000058
:10009000F5110000F5110000F5110000F511000048
:1000A000F5110000F5110000F5110000F511000038
:1000B000F5110000F5110000F5110000F511000028
:1000C000F5110000F5110000F5110000F511000018
:1000D000F5110000F5110000F5110000F511000008
:1000E000F5110000F5110000F5110000F5110000F8
:1000F000F5110000F5110000F5110000F5110000E8
:10010000F5110000F5110000F5110000F5110000D7
:10011000F5110000F5110000F5110000F5110000C7
:10012000F5110000F5110000F5110000F5110000B7
:10013000F5110000F5110000F5110000F5110000A7
:10014000F51100002DE9E04F2746A046A146A24642
:10015000A346A446A2B02DEC000A84F300882546ED
:100160002646A4473DEC000A22B0BDE8E08F00001F
:100170007BB972B90029BEBF00204FF0004106E0F4
:1001800008BF00281CBF6FF000414FF0FF3000F0A7
:10019000AFB9ADF1080C6DE904CE002909DB002BE5
:1001A0001ADB00F035F8DDF804E0DDE9022304B0E5
:1001B0007047404261EB4101002B1BDB00F028F847
:1001C000DDF804E0DDE9022304B0404261EB4101C7
:1001D000524263EB43037047524263EB430300F028
:1001E00017F8DDF804E0DDE9022304B0404261EBDA
:1001F00041017047524263EB430300F009F8DDF818
:1002000004E0DDE9022304B0524263EB430370478C
:100210002DE9F0478C46089D04468A46002B4AD1BA
:100220008A42174662D9B2FA82F64EB1C6F1200E62
:1002300001FA06F3B740B44020FA0EFE4EEA030A74
:100240004FEA1748230C1FFA87F9BAFBF8FE08FBA0
:100250001EAA0EFB09F243EA0A439A420BD9FB1885
:100260000EF1FF312CBF012000209A4202D9002854
:1002700000F02A818E469A1AA3B2B2FBF8F008FB6E
:10028000102200FB09F943EA0244A14507D93C19B1
:1002900000F1FF3302D2A14500F210811846A4EB11
:1002A000090440EA0E4000211DB1F4400023C5E9D5
:1002B0000043BDE8F0878B4208D9002D00F0F280A2
:1002C0000021C5E9000C0846BDE8F087B3FA83F1C8
:1002D00000294ED16345C0F0E880824240F2E580BB
:1002E0000846002DE5D0C5E9004AE2E702B9FFDE85
:1002F000B2FA82F6002E40F099808B1A4FEA124E25
:100300001FFA82F801214FEA144CB3FBFEF20EFBF8
:10031000123008FB02F94CEA004CE14508D917EB12
:100320000C0C02F1FF3302D2E14500F2CA801A46FA
:10033000ACEB090CA3B2BCFBFEF00EFB10CC08FB2F
:1003400000F843EA0C44A0450ED93C1900F1FF33F4
:100350002CBF4FF0010C4FF0000CA04503D9BCF1AD
:10036000000F00F0A8801846A4EB080440EA024001
:100370009AE7C1F120048B4002FA01FE0CFA01F663
:10038000E24020FA04F72CFA04FC00FA01F81343C7
:100390003E431F0C320C1FFA83F9BCFBF7F007FB3E
:1003A00010CC00FB09FA42EA0C4CE24508D913EBE9
:1003B0000C0C00F1FF3202D2E24500F289801046B7
:1003C000ACEB0A0CB6B2BCFBF7FA07FB1ACC0AFB83
:1003D00009F946EA0C42914506D99A180AF1FF3606
:1003E00001D291457AD8B2464AEA0040A2EB09020E
:1003F000A0FB0E67BA42B446B94602D307D1B04556
:1004000005D2B6EB0E0C67EB030301389946002DBD
:100410006BD0B8EB0C0362EB090202FA04F4CB4098
:10042000CA4000211C43C5E9004242E7B740C6F17B
:10043000200201FA06F3B44021FA02FC4FEA174EFB
:1004400020FA02F21FFA87F8BCFBFEF11A430EFBFA
:1004500011CC01FB08F0130C43EA0C4C604507D9A2
:1004600017EB0C0C01F1FF3301D2604533D819466C
:10047000ACEB000C92B2BCFBFEF00EFB10CC00FB10
:1004800008F342EA0C4C634507D917EB0C0C00F15A
:10049000FF3201D2634525D81046ACEB030340EA96
:1004A000014130E72946284603E7841A6CEB030331
:1004B00001209A4615E702383C4455E702383C448F
:1004C000EDE6023ABC4433E7AEF1020E3B44D2E61D
:1004D00002389C4474E70239BC44C9E7AAF1020A15
:1004E0001A4481E70238BC44D7E72946E1E600BF59
:1004F000704700BF830003F1A04303F54053D3F8D6
:10050000002810B4002A1BDAD3F8002802F00302F6
:10051000022A05D0D3F8002802F00302032A0FD1E3
:10052000012100F01F04A1404209074C203244F889
:100530002210BFF34F8FBFF36F8F044AC3F8002818
:10054000002110BC01F0A0B800E100E00001008033
:100550008FB5584800F048FB002440F21717564E5C
:10056000564D04F5C073214646F8237028460134E1
:1005700000F03AFB082CF4D140F207174E4E504DD4
:1005800004F5C073214646F823702846013400F074
:100590002BFB202CF4D14B4800F026FB002440F22A
:1005A0001717454E484D04F5E073214646F8237071
:1005B0002846013400F018FB082CF4D140F207174C
:1005C0003D4D424E04F5E073214645F82370304618
:1005D000013400F009FB202CF4D100243C4800F049
:1005E00003FBC5F8C0444FF480250520FFF782FFC8
:1005F0001520FFF77FFF2A20FFF77CFF3920FFF748
:1006000079FF3A20FFF776FF4220FFF773FF312092
:10061000FFF770FF0920FFF76DFF0A20FFF76AFF61
:100620001C20FFF767FF1D20FFF764FF2C20FFF75A
:1006300061FF0A20FFF75EFF0B20FFF75BFF2968D1
:10064000244800F0D1FA10222146684601F0AAF9A8
:100650002B6868460093029500F042F8012000F0F4
:100660006FF8204600F058F8204600F07DF8012190
:10067000204600F08DF8184A1848D2F88C3043F420
:100680004063C2F88C304FF004131C6800F0ACFAE1
:100690000820FFF72FFF24F00104BFF34F8FBFF3B3
:1006A0006F8F640864002046214622462346FFF7E8
:1006B00049FD00BF5C2D0000003000507A2D000085
:1006C000A52D0000DA2D0000F72D0000272E0000D8
:1006D0005B2E00007F2E000000ED00E0972E000052
:1006E00082680C4B9A60036883F38888436883F3BD
:1006F0008988027B02F00101EFF3948323F0030366
:10070000920748BF43F0020309B143F0010383F3AA
:100710009488704700ED02E0084AD36848B123F49A
:1007200000531B041B0C43F0BF6343F40033D3603E
:1007300070479BB243F40053F5E700BF00ED00E0C3
:10074000084AD36840B19BB243F4804343F0BF638F
:1007500043F40033D360704723F480431B041B0C25
:10076000F4E700BF00ED00E0084AD36840B19BB257
:1007700043F0080343F0BF6343F40033D360704792
:1007800023F008031B041B0CF4E700BF00ED00E09E
:10079000084B1A6818B142F001021A60704722F043
:1007A00001021A601A6811B142F00202F5E722F064
:1007B0000202F2E7D0ED00E008B504460846114613
:1007C0001A46A04701F06AFF01F012F870B50C2537
:1007D0004D43C66890F90B0074198842A8BF2146A2
:1007E0004FF0200492FBF4F4B8BF715902F01F00DF
:1007F00001EB8401196070BD07B501ABFFF7E6FF9F
:100800000123019A03FA00F013680343136003B055
:100810005DF804FB2DE9F8430446FF2200214FF068
:100820000C0E4368058900685D4394F80AC02844AB
:10083000E2728C4505DC00252389AB4222DCBDE851
:10084000F883B5FBF3F20EFB01F7D4F80C801F2AF6
:1008500008EB0706C8BF1F324FEA930306F10409ED
:10086000C8BF520903F10303C6E9019923F003034A
:10087000D4BFE17248F8070001F10101C8BF00EBE5
:100880008200D6E76268E3686A4320681E1D81180B
:1008900086509A6820464A609A68116099602A4694
:1008A0000021FFF7A9FF0135C6E7002070470000CF
:1008B0000B6801330B60014B1B681847900E00203A
:1008C0002DE9F04F85B00E9C9B46012CB8BF01244A
:1008D000012B0CBF30232023154680468946012674
:1008E0000A270022DFF870A0019402930AF10104A4
:1008F0000AB9AA451ED2B5FBF4F049463030C047CC
:1009000001220136B5FBF4F10A23013F012F04FB5C
:100910001155BAFBF3FAE9D1494605F13000C04759
:10092000BBF1030F03D1019B9C1B002C0FDC05B016
:10093000BDE8F08F019BBB42E4DBBBF1020FE1D8C5
:100940004946029803920136C047039ADAE74946BE
:100950002020C047013CE8E7FFC99A3B014B1860E3
:10096000704700BF900E00202DE9F04F4FF0000AB5
:1009700006460F464FF0FF39D04689B01C46531E3D
:100980000493002505E06DB9252800F01181394652
:10099000B047049B13F8010F04930028F3D109B06A
:1009A000BDE8F08F642861D019D839280AD83128D9
:1009B00050D22D283CD030283DD0252808D13946AA
:1009C000B047DEE7582800F08880632800F0EA800E
:1009D00039462520B047049B39461878F0E770283F
:1009E00071D006D8692841D06C283CD06828D0D076
:1009F000EEE7752857D017D87328E9D1236804F19A
:100A0000040B1C46254615F8010B002840F0BF805A
:100A1000B8F1030F40F0D580E41AA9EB0404002CD0
:100A200000F3BB805C46ACE7782856D07A28DEE736
:100A30004FF00308ADE7B9F1000F0EDAB8F1000F7F
:100A400000F0BC80A0F13009B8F1000F08BF4FF0F2
:100A500002089EE7B9F1000FF4DB0A2303FB090942
:100A6000A9F13009F0E70AF1010A92E7BAF1010FA2
:100A7000C5BF073424F0070325681D68D4BF0434BC
:100A800003F10804002D05DA39462D20B0476D42E8
:100A900009F1FF3943462A46CDF8009039463046E1
:100AA000FFF70EFF6DE7BAF1010FC5BF073424F061
:100AB000070322681A68CCBF03F108040434CDF898
:100AC00000904346EAE739463020B047394678205F
:100AD000B0474FF008094FF001080822BAF1010FA2
:100AE000C5BF073424F00703236803F10804CABF15
:100AF0001B68059305934FF000039346D8BF043459
:100B0000039307930BF1FF3B059B4FEA8B0023FAFE
:100B100000F010F00F0009D1079B13B9BBF1000FD3
:100B200024D14FF0300C07E0069AEBE709288CBF80
:100B30004FF0570C4FF0300C394660440692B047E6
:100B4000039B079501330393BBF1000FECD1B8F180
:100B5000030F7FF416AF039BC3EB4905002D7FF70E
:100B600010AF39462020B047013DF7E7531E9145AD
:100B70000693E9DBB8F1010F03D139463020B047C5
:100B8000E2E7B8F1020FDFD139462020F7E7394616
:100B900003932C46B047039B34E739462020B047E7
:100BA000013C3CE72068251D3946B0472C46E8E665
:100BB000AA46A8464FF0FF390125EAE64FF00108A2
:100BC000E7E65C460546E4E6002313B502AC44F8CC
:100BD000043D02460B4603482146FFF7C5FE02B01E
:100BE00010BD00BFB10800000FB407B504A951F84B
:100BF000040B0191FFF7E8FF03B05DF804EB04B0CC
:100C00007047704710B54FF02003EFF3118483F362
:100C1000118800F011F80122054BC3F840254FF070
:100C2000FF32044B9A62DA6284F31188002010BD0F
:100C30000090035000ED00E0484A136843F00203BF
:100C400013600022D30003F57F03D3F800130131B2
:100C500008D0D3F800130132D3F80433B2F5807F03
:100C60000B60EFD13E4AD36913F001033BD03D4BFB
:100C70001946D3F80024012AFBD1C3F80425D1F882
:100C80000034012BFBD1364BDA69D20708D5DA697B
:100C9000344922F00102DA61D1F80024012AFBD1A3
:100CA0001A6A01320AD11A6A22F0FF0242F02002C7
:100CB0001A622C4AD2F80034012BFBD10022294BB6
:100CC000C3F80425D3F80024012AFBD1BFF34F8FCA
:100CD0002549264BCA6802F4E0621343CB60BFF398
:100CE0004F8F00BFFDE7126A0132C0D0204A116861
:100CF00009290AD11F490968013901299EBF4FF00E
:100D00005021C1F81431C1F818311368092B09D1E9
:100D1000184B1B68012B01BF174A1360A2F638223B
:100D2000C2F87835124B1B68092B0BD1114B1B688D
:100D3000022B07D10022104B1A600122A3F63823A0
:100D4000C3F87825084AD2F88C3043F44063C2F8DF
:100D50008C300A4B0A4A1A60704700BFD0ED00E0A1
:100D60000080FF000090035000ED00E00400FA0551
:100D70003001FF003401FF00384A0050940E00207B
:100D80000090D0030A2838B50446074D04D12868DE
:100D90000D2143685B6898472868E1B243685B6847
:100DA0009847204638BD00BF000000200148FFF7EB
:100DB000D5BD00BF850D000008B5044801F0FCF961
:100DC000034B1860FFF7F2FF002008BD032F00005F
:100DD0000000002010B54FF02003EFF3118283F3E1
:100DE0001188114C237823B982F311886FF04400E5
:100DF00010BD013BDBB2237023B182F311886FF089
:100E00000F00F5E7094B0121187828B1217082F312
:100E100011886FF00A00EBE7197082F31188044A19
:100E200011601870E4E700BF0600002005000020F4
:100E30000450005010B54FF02002EFF3118382F3FD
:100E40001188124C207888B183F311884FF050221A
:100E5000D2F81C34D2F8182403F0030343F480338F
:100E6000934314BF6FF04300002010BD0122227095
:100E700083F311884FF05023C3F80401C3F8181509
:100E80000221C3F804139A60E0E700BF04000020C9
:100E90004FF0502330B5D3F80851D3F80423D3F8DA
:100EA000004102F00102D3F80413D3F8040115B194
:100EB0000025C3F80851B4B14FF050230024C3F803
:100EC000004122B14FF050230122C3F8082348B15A
:100ED00000224FF05023C3F804218A0702D50222D2
:100EE000C3F8082330BD002AF1D04FF05023D3F8C7
:100EF0000C3403F00113B3F1011FE8D1E2E708B5A8
:100F000000220121052000F0A5FB052000F07EFB5A
:100F1000002008BDF8B54FF02002EFF3118382F3F3
:100F20001188264A1078441C147070B183F311881C
:100F30004FF05023D3F80C3403F00113B3F1011F29
:100F40000CBF00206FF0430007E01D4D2F782FB13C
:100F5000107083F311886FF00A00F8BD01262E701F
:100F600083F311884FF0502421B3052000F05EFB7D
:100F7000C4F80071D4F80433C4F804632660D4F8CC
:100F800000219AB10022DB0758BF0123C4F80021D9
:100F90004FF0200258BFC4F808330A4B0520C3F8AD
:100FA000802100F033FB00232B70C1E720BF40BF3E
:100FB00020BFE4E7C4F800112660F4E70600002033
:100FC0000500002000E100E070474FF02003EFF340
:100FD000118083F31188704700230D4A10B5C2F8C1
:100FE0004031FFF7F2FFD2F8043540F247120949C9
:100FF0000C681B1B23F07F43B3FBF2F302FB03429D
:101000000A6080F311881846BDE8104001F0DCBC8E
:10101000005001500800002038B51B4801F0CCF802
:1010200070B3436801211B689847002440F24713BE
:10103000164D4FF40012C5F80845C5F840354FF479
:101040008033C5F84433C5F80433114B01211C60CB
:10105000104B1520C3F88021224600F0FBFA152022
:1010600000F0D4FA012320460B4A13602B60D5F818
:10107000043503F2471323F07F43C5F8403538BDEC
:101080004FF0FF30FBE700BF242F0000005001505D
:101090004051015000E100E00850015070B54CF69D
:1010A0006905B0F1FF3F14BF02462A46FFF78DFFE6
:1010B000124B134C1E68531EAB42A8BF2B4640F286
:1010C0004715D4F8041523EAE3738A1B22F07F4204
:1010D00002F5A37205FB0323B3FBF5F305FB0363E2
:1010E000591A21F07F411F2998BF5B1923F07F43D4
:1010F000C4F8403580F3118870BD00BF080000209F
:101100000050015008B5FFF760FF084B084AD3F8BC
:10111000043512689B1A40F2471223F07F43B3FB59
:10112000F2F380F31188184608BD00BF005001504B
:101130000800002004488168406A884203D00349BF
:101140004FF080520A6070472001002004ED00E05B
:10115000202080F311880D498A684FF02800104440
:10116000EFF3098C80E8F01F094F4FF000664A6AE0
:101170008A603E60506E0023536680F3118802F14E
:10118000280090E8F01F8CF30988704720010020A8
:1011900004ED00E01EF0040F0CBFEFF30880EFF346
:1011A0000980816931F8021C11F0FF010229FFD08A
:1011B00000B500F0EDFA00BD014910220A60704749
:1011C00010ED00E0404080F3118830BF704700BF51
:1011D000404080F311884FF004007146014202D074
:1011E000EFF3098001D1EFF30880714600B500F0FC
:1011F0006FF900BD00B572B60B4A106A00281EBF19
:101200000021116200F0FEFF62B6EFF30580A0F14D
:1012100010004FEAC0000549014409C998475DF82C
:1012200004EB03480047000020010020BC2A000016
:1012300035110000002320210348C2180133412B3F
:1012400082F80013F9D1704700E100E0084A09492B
:10125000936809685866996607494B6843F080535C
:101260004B60002383F311889368986E704700BF2A
:1012700020010020FC34000000ED00E038B5194CDE
:1012800005461948FFF7B0FCA36AD90602D51748EE
:10129000FFF7AAFCA36A1A0702D51548FFF7A4FCBA
:1012A000A36A9B070ED51348FFF79EFC616BA36AE8
:1012B000180607D51048FFF797FC1DB1A36A23F065
:1012C0008003A362074CA26AD20702D50B48FFF73E
:1012D0008BFCA36A9B0602D50948FFF785FC00201A
:1012E00038BD00BF00ED00E0D8300000EF30000056
:1012F00001310000153100002E31000045310000A1
:101300006531000038B51E4C05461E48FFF76CFCE1
:10131000A36AD80409D51C48FFF766FC184A0020C8
:10132000936A43F47F43936238BDA36A190501D5DC
:101330001648F1E7A36A9A0514D51548FFF754FC3F
:10134000A16BA36A1B0407D51248FFF74DFC1DB122
:10135000A36A23F40043A362094B9B6A5805DDD5B9
:101360000D48D9E7A36A5905FAD4A36ADA0501D56D
:101370000A48D1E7A36A9B04D0D50948CCE700BF4F
:1013800000ED00E0442F0000EF30000001310000CC
:101390005B2F0000752F00008B2F0000A72F00008F
:1013A0006531000010B51C4C1C48FFF71DFCA36AFA
:1013B0009A0102D51A48FFF717FCA36ADB0102D590
:1013C0001848FFF711FCA36ADC0202D51648FFF7A4
:1013D0000BFC114CA36A180302D51448FFF704FC58
:1013E000A36A590302D51248FFF7FEFBA36A9A03CA
:1013F00002D51048FFF7F8FB074CA36ADB0302D5C0
:101400000D48FFF7F1FBA36A00206FEA03436FEA80
:101410001343A36210BD00BF00ED00E07532000071
:101420008E320000A2320000BD320000CF32000038
:10143000EE320000143300002F33000010B51A4CB8
:101440001A48FFF7D1FBA1696369580602D518480D
:10145000FFF7CAFB6369D90707D51648FFF7C4FB36
:10146000636943F0FF03636110BD63699A0701D5A7
:101470001148F3E763695B0701D51048EEE763693C
:10148000180701D50E48E9E76369D90601D50D486B
:10149000E4E763699A0601D50B48DFE763691B0639
:1014A000DED50A48DAE700BFD0ED00E09531000054
:1014B000AF310000C0310000D7310000F63100002C
:1014C000123200003032000046320000613200006B
:1014D0003B4B70B55D6801F07F43B3F17F4F04462D
:1014E0000E4618D1CA0716D54B061FD40168354BD6
:1014F0000B44012B98BF016C3348FFF775FB16F0C6
:10150000080F2F4B0DD0EFF389845B6818050DD4BD
:101510002E48FFF769FB2146BDE87040002000F02F
:1015200005B9EFF388845B681905F1D4C5F30805A4
:10153000EA1E092A39D8DFE802F0053234282F38AC
:10154000383838362248FFF74FFB1D4BDA6A9207CE
:1015500001D52048DDE7DB6A5B00DCD51E48FFF7DC
:1015600043FB1E4B1B782BB10120FFF787FE06289B
:10157000D1D170BD1A4B1B781BB10120FFF7C2FE01
:10158000F5E7184B1B889BB213B1FFF70BFFEEE793
:10159000154B5B69002BBED0FFF750FFBBE7002067
:1015A000E3E70020EAE71148B3E711481149A5F144
:1015B00010020F2DD8BF01460F48FFF715FBAAE711
:1015C00000ED00E0A6ED0501EE2F00000E3000005A
:1015D000333000004B3000006D30000028ED00E09B
:1015E00029ED00E02AED00E0D0ED00E08D300000B4
:1015F000C02F0000D52F0000C4300000024A5369FC
:1016000043F010035361704700ED00E043B2002B3C
:1016100008DB012200F01F0002FA00F0024A5B0919
:1016200042F82300704700BF00E100E043B2002B06
:101630000DDB012200F01F0002FA00F05B09044AF2
:10164000203342F82300BFF34F8FBFF36F8F7047F3
:1016500000E100E043B2002B01F10101A8BF03F15A
:1016600060434FEA4111B8BF054BC9B2ABBF03F5A8
:10167000614300F00F0083F800131954704700BF56
:1016800014ED00E0FFF7A4BD43B2A9B1002B12DBBB
:1016900001215B099B0003F1604303F56143D3F82B
:1016A000802200F01F0001FA00F022EA0000C3F8D7
:1016B0008002D3F880327047002BFCDB01225B09EB
:1016C0009B0003F1604303F56143D3F8801200F0FF
:1016D0001F0002FA00F00843E9E70000F8B51646DB
:1016E0000C461F4604220A9B0999054601F0C0F8E2
:1016F0000023A6F120010C4A214421F0070122F029
:101700000102C5E91333C5E916468A61069A0F60DE
:101710004A60079A8A60089ACA604FF08072CA616C
:10172000A9646B66F8BD00BFB907000038B5044670
:101730000D4605281AD8DFE800F00319191315170C
:101740000D48FFF751FA00F0A9FFAA6901460B48BE
:10175000FFF74AFA29462046BDE8384000F01CB899
:101760000748EEE70748ECE70748EAE7014607487D
:10177000FFF73AFAE7E700BF5B330000F9330000F8
:101780007B330000A1330000BB330000D6330000E0
:1017900001460068FFF7CABF052810B50CD000F05D
:1017A000AFFF60B100F0ACFF0C490D4B002808BF43
:1017B00019460C48FFF718FAFFF704FDFCE700F0A4
:1017C000AFFF0028EED1084C0848A168FFF70CFADB
:1017D000A068BDE8104000F00BB800BF3534000031
:1017E000393400004A340000200100206A3400002F
:1017F00038B505464FF02003EFF3118483F31188C9
:1018000000F0C8FF0A4B9B68AB420BD1094B5A68EA
:10181000C2F3080212B92046FFF718FD5A6842F0D9
:1018200080525A602046BDE8384000F05BBE00BFE1
:101830002001002000ED00E0202080F31188064800
:101840004FF40061401880F30988022080F3148867
:10185000BFF36F8F00F006F89006002030BFFFF74F
:10186000FDBF00BF08B5084B084A23F07F03936013
:10187000BFF34F8FBFF36F8F00F0DEFC00F0E6FC8C
:10188000FFF7D8FC00F006FD0000000000ED00E0CE
:1018900008B5FFF7E3FFBDE80840FFF74BBC0000C9
:1018A0000522034B5A60BFF34F8FBFF36F8F704712
:1018B00090ED00E0BFF35F8F0022014B5A6070474C
:1018C00090ED00E0184919480B6870B50468C3F33F
:1018D00007239C4225D8FFF7EDFF4FF6AA73426815
:1018E00000200B63844202F1100603D1FFF7D8FFFA
:1018F000002070BD157A56F8103C05F01F0223F049
:101900001F031A4356F8043C6D0923F01F0343F0EC
:10191000010343EA45038860CA6001300B61324627
:10192000E0E74FF0FF30E4E790ED00E0CC2E000060
:101930000138013910F8013F11F8012F934202D10B
:10194000002BF7D11A46981A7047F0B581EA0004C7
:10195000A50703460BD0013B0A4491421DD1F0BDBF
:10196000002AFCD011F8014B013A03F8014B9C0707
:10197000F6D10C461D1F8F183E1B032E08D86FF0A2
:101980000305940805FB0422A40023442144E2E754
:1019900054F8046B45F8046FEEE711F8014B03F8B7
:1019A000014FDAE70346F0B5C9B29C070FD11D46D7
:1019B00041EA012444EA04449F187E1B032E0CD8FC
:1019C000940803EB840413449C4209D1F0BD002A1F
:1019D000FCD003F8011B013AE7E745F8044BECE7BC
:1019E00004F8011BF0E70000074B03EB8000D0F880
:1019F000003223F44033C0F80032D0F8003243EA1A
:101A00000141C0F80012704700258450F8B5036802
:101A100001F01F049B680D461B79494944EA4314B1
:101A20000023D1F804238668D2B203F5A27051F8DE
:101A30002000C0F30420844267D122FA03F0C007DB
:101A400063D59A0002F1A04202F55042D2F8100587
:101A500020F00100C2F81005012202FA03F3C1F8D8
:101A6000083320460021FFF7BFFFB068E84010F0C0
:101A7000010049D0F068E84010F0010044D07069DE
:101A8000E84010F001024CD0B369EB40DB0740D4D2
:101A9000336923FA05F2F36923FA05F505F0010528
:101AA00002F00103AB420CBF022501250021244EA8
:101AB00001F5A27356F8230010F003002BD18B0020
:101AC00003F1A04303F55047D7F81025240222F470
:101AD000473222F44072C7F81025D7F8102504F4D5
:101AE000F85444EA054503F551431543C7F810552A
:101AF0001860D7F8103543F00103C7F810350123FB
:101B000003FA01F1C6F80413F8BD0133082B8CD198
:101B1000A7E70325CAE701310829C9D16FF01200F0
:101B2000F2E7F169336920464B4023FA05F515F0D9
:101B3000010F0CBF03210221FFF756FF1046E3E718
:101B400000D0005010B504688068A468012924689A
:101B5000C06903D158406060002010BD00334FF0D1
:101B6000010118BF0123D04000F0010091408342E1
:101B700014BFA160E160EFE770B504688068A468F5
:101B8000C069256801296E692C696D6880EA0400C6
:101B900084EA050404EA060480EA04001CBFD0407D
:101BA00000F001001860002070BD8368186872B1F1
:101BB00008605A68196002B95960002070471060C7
:101BC0005868814208BF5A600DE00246006800284C
:101BD000F3D08842F9D10868002AF0D15A68186019
:101BE000914200D1586000230B60E6E701292DE9FE
:101BF000F04118BFD4B2064612BF25461F25002467
:101C00004FF001088768AC4202D90020BDE8F0819E
:101C1000FB6808FA04F223EA0203FB60214630461F
:101C2000FFF7F4FE0028F1D10134E4B2EBE7000045
:101C300008B5094B1A786AB901210D2019700521E0
:101C4000FFF708FD0D20FFF7E1FC4FF00042034BCA
:101C5000C3F80423002008BD0C00002000D0005071
:101C60002DE9F74F8046856803F47040B0F5804F4A
:101C70001E4649D02CDCB0F5805F3DD0B0F5405F0A
:101C80003ED060BB06F44077B7F5807F3ED0A7F525
:101C9000007463426341012919BFD4B2A1464FF0D9
:101CA0001F0900244FF0010B06F0010C4FEA4C070E
:101CB00047EA0C0747EA0020DFF8C8A040EA83079C
:101CC00006F00203A14523D2002003B0BDE8F08F47
:101CD000B0F5E04F16D005DCB0F5A04F0ED06FF098
:101CE0001500F2E7B0F5404F04D0B0F5504FF6D1F3
:101CF0000720C7E70620C5E70120C3E70320C1E7A7
:101D00000420BFE70520BDE70220BBE70323C2E7AD
:101D1000D8F800209268117904F01F0242EA4112BB
:101D200080324AF82270A9680BFA04F2002B25D001
:101D30001143A9606969B0064CBF114391436961C1
:101D4000A96970064CBF11439143A96129697007C5
:101D50004CBF114391432961E96930064CBF0A43E6
:101D600021EA0202EA61214640460193FFF74EFE56
:101D70000028AAD10134E4B2019BA3E721EA0201C1
:101D8000D7E700BF002584502DE9F843444E35685D
:101D9000012D59D12F464FF00009424A936812682D
:101DA000DC69D2F80880D3E902120A40D3E90510B1
:101DB000014322EA0102D8F800101B6909695C405E
:101DC0004C4022EA040472BB3260002301279C4687
:101DD000354ED6F8042307FA03F1114211D003F16E
:101DE000A05202F5515292001168012909D103F560
:101DF000A27056F82000C2F800C0C0F30420814051
:101E00000C430133082BE4D104B3264FBB681E6892
:101E1000E6B1B3681C4204D07368224631463846A6
:101E200098473668F4E73A420AD098F8043009F047
:101E30001F00002140EA4310FFF7D6FD22EA070207
:101E400009F101097F00BEE70024BEE7012D0DD195
:101E50000026144B9C681B689F68D4E902321A4024
:101E6000D4E905310B4322EA03020AB9BDE8F8833D
:101E7000154212D0E169236997F804C04B40F34042
:101E800013F0010F06F01F000CBF0321022140EAEE
:101E90004C10FFF7A9FD22EA050201366D00E4E7C8
:101EA0007CD10050240F002000D0005001292DE9E2
:101EB000F04118BFD4B2064612BF25461F250024A4
:101EC0004FF001088768AC4202D90020BDE8F081DC
:101ED000FB6808FA04F21343FB6021463046FFF723
:101EE00095FD0028F2D10134E4B2ECE770B54B79EE
:101EF000012B23D18B79032B20D1CC792CB1012C50
:101F00001CD103689B681B79C3B10A7912B1022AFC
:101F100014D10E2247F6122603689B681D680B68D1
:101F2000B3426BD027D8B3F5965F61D012D8B3F522
:101F3000167F4DD005D8B3F5967F74D06FF0220090
:101F400052E0B3F5966F50D0B3F5166FF6D14FF45B
:101F50001D233FE0B3F5615F4CD004D8B3F5165FA5
:101F6000ECD1324B36E0B3F5964F45D0B3F5E14FA7
:101F7000E4D12F4B2EE0B3F5E13F48D012D84DF617
:101F8000C026B3423DD005D8B3F5164FD6D14FF495
:101F90001D031FE0B3F5614F36D0B3F5963FCDD1A9
:101FA000244B17E0B3F5E12F37D008D8B3F5613FE4
:101FB00030D0214EB342C1D14FF080630AE0B3F577
:101FC000612F2DD01D4EB342B8D14FF0805301E0A8
:101FD0004FF41C33C5F824358368224303C9C5F880
:101FE0006C2583E80300002070BD4FF49E23F1E7C9
:101FF000134BEFE7134BEDE7134BEBE74FF4000305
:10200000E8E74FF46503E5E74FF46B03E2E74FF0D1
:10201000EB73DFE74FF06C73DCE74FF0E863D9E771
:102020004FF07063D6E74FF4A033D3E7005027009A
:1020300000C0750000903A0190D0030040420F00AC
:1020400000B0130000F03A0000A04E000B4682687A
:1020500092E8030083E80300002070470368826869
:102060009B681B68D3F8100138B1127A00200A70FF
:102070000122C3F810011A6070474FF0FF3070471B
:1020800082B002AA02F8011D002103689B681B6848
:10209000C3F82011C3F844250122C3F848259A60EB
:1020A000D3F820110029FBD0DA6002B07047036832
:1020B0009B681B68D3F8240118B1D3F88004C3F8D7
:1020C000800470472DE9F04101264FF0030E4FF0D8
:1020D000000C03680A689B6806FA02F71C681B4B31
:1020E00085689F6002F1800743F827E04F6807F199
:1020F000800843F828C0C4F80C25C4F814758F680C
:102100007A1C10D0CA68511C0DD002F18001964093
:102110009E6043F821E007F1800143F821C0C4F834
:102120000825C4F810752946FFF7E0FE58B90823C2
:10213000C4F800351D440123C4F81001C4F8345517
:10214000C4F838352360BDE8F08100BF0025845015
:1021500030B585B005466C46044B0FCB84E80F00C4
:1021600021462846FFF7AEFF05B030BD3C2D0000EC
:1021700030B585B005466C46044B0FCB84E80F00A4
:1021800021462846FFF79EFF05B030BD4C2D0000CC
:1021900038B5084B53F82040013053F82050204602
:1021A000854204F10C0400D838BD54F80C3C5B683F
:1021B0009847F4E7E8340000104B70B505461E461A
:1021C0000F4C9C4204D10E4CB44209D1002412E0C1
:1021D00062681AB122681268AA420CD00C34F0E787
:1021E00063680BB90C34EFE7236828461968FFF7DA
:1021F0009FFB0028F6D1204670BD00BF300F0020A5
:10220000B80E0020FEF7E0BE08B50A4D4FF02002E0
:10221000EFF3118382F3118800F06CFB0121044677
:102220000228D8BF084600F01BFC2C62FEF7CAFF4C
:10223000ECE700BF200100200248034A0021121AE7
:10224000FFF7B0BB00000020500100200248034A05
:102250000349121AFFF779BB900E0020440F0020AB
:102260004035000008B50220FFF792FF0748FEF74F
:10227000BBFC0320FFF78CFF00F0ACFAFEF768F917
:10228000034A137B23F00103137308BD10350000CC
:102290009C00002080B586B0374B06AF83F30888DA
:1022A0000024E022354B364D83F82220DC771C7663
:1022B0005C769C76DC765A6A324E42F4E0225A62B0
:1022C0005A6A42F400225A629C63DA6892B242F07F
:1022D000BF6242F40832DA60FFF790F9FEF76CFF54
:1022E0002046FFF755FF0120FFF752FF00F0CAF923
:1022F000254B756205930123CDE90144CDE90343E4
:102300000094224B4FF480622149284600F028FABD
:102310006B7B344623F0040213F01B0F6A7305D164
:102320002B6A013302D1284600F02EF9194B012205
:1023300005930F23CDE903320023174ECDE9013376
:1023400000934FF4A072154B1549304600F008FA7F
:10235000737BE66023F004037373124BA560C4E93A
:1023600006330A4A104B114C83F3098863B60021E7
:1023700081F3118810462047900E002000ED00E008
:102380009C00002020010020003500006522000094
:102390005001002005350000300000200922000017
:1023A000500500203801002050050020B90700002A
:1023B000D0E900231A6002685360704708B5FEF741
:1023C000A1FE054B054A1B68002118441061184600
:1023D000BDE8084000F044BB0C01002020010020B3
:1023E0004FF02003EFF3118083F311887047000052
:1023F00038B5104C234653F8285F9D4200D005B9EC
:10240000E568A36878B973B15A7BD2060BD11A6A12
:10241000013208D1DA897F2A05D9074A1268934226
:1024200001D0636238BDAB4201D0FFF7C7FF6562E0
:10243000F8E700BF200100200C350000F8B50D467C
:102440000746FFF7CDFF4FF4004600220021044667
:10245000094B0A481A61C6FB07014FF4A02200236A
:10246000FDF786FE064B1860064B1D60FFF7A6FFC2
:1024700084F31188F8BD00BF20010020FFFF040095
:102480000C0100200801002010B50146FFF7A8FF4D
:102490004B7B04465A060DD50846FFF789FF4B7B58
:1024A00023F040034B73054B9868431A5842584138
:1024B000FFF79EFF84F3118810BD00BF20010020AC
:1024C00010B50146FFF78CFF04460846FFF770FF82
:1024D0004B7B23F002034B7384F3118800238B6042
:1024E00010BD0000EFF305830D2B0BD81BB1074B7C
:1024F0005B681B0506D5064B9A685B6A9A4201D059
:10250000FEF7A4BE80F31188704700BF00ED00E025
:102510002001002010B5FFF763FF0A4B04469A68BC
:102520000120D37B0133D373FFF762FF84F311885B
:102530004FF02003EFF3118083F31188BDE81040C2
:10254000FFF7D0BF20010020036810B5984213D0D8
:1025500093B191F90E2093F90E40944206DD5A682A
:10256000C1E900325A681160596010BD4468A34245
:1025700002D01B68002BEED1436808604B604368B3
:1025800019604160F1E7000038B50446FFF728FF05
:10259000214605460648FFF7D7FF637B002043F03E
:1025A00040036373FFF724FF85F3118838BD00BF34
:1025B00048010020427BD20604D1036A013301D1D5
:1025C000FFF7E2BF704738B550F8103C0446A0F161
:1025D000180513B12846FFF773FF14F80B3C284683
:1025E00023F0040304F80B3CBDE83840FFF7E2BFDA
:1025F00070B50446FFF7F4FE0B4D06462046FFF784
:10260000D7FE21462846FFF79FFF637B55F8200C35
:1026100043F040036373031B58425841FFF7E8FE41
:1026200086F3118870BD00BF48010020114B10B522
:102630001B68EBB110498B68DA897F2A18D80F4ADA
:1026400093F90E401268944212DB0D4A12689342CD
:102650000ED01A6A01320BD10A69824206DC184692
:10266000FFF7C6FFBDE81040FFF7A8BE121A0A61C7
:1026700010BD00BF0C010020200100200801002037
:102680000C3500000021044B084603F12802C3E981
:102690000A22FFF7D3BE00BF20010020014B98683B
:1026A000704700BF20010020F8B505460F464FF0E7
:1026B0002003EFF3118483F311884FF400460021C7
:1026C000084800234FF4A022C6FB0701FDF750FD88
:1026D0000549421C05F1180000F03AF984F311880D
:1026E000F8BD00BFFFFF0400C7250000427BD206F3
:1026F00004D1036A013301D1FFF746BF70470000E0
:10270000EFF305800D2807D838B1044B586880F4E2
:102710000060C0F3C02070470120704700ED00E06A
:10272000024B9B68187B00F00100704720010020DD
:1027300010B54FF02003EFF3118483F31188437B2E
:10274000590702D484F3118810BD23F004034373A6
:10275000FFF7CCFF2046BDE81040FFF7C3BE0000E6
:1027600030B587B00E9D044604950D9D03950C9DD4
:1027700002950B9D01950A9D0095FEF7AFFF044B56
:102780009B6813B9236607B030BD1B6EFAE700BF24
:1027900020010020036D10B5044603B19847637B08
:1027A000DA060AD1226A013207D12046FFF76CFE11
:1027B000637B43F00803637310BD9B0702D520467B
:1027C000FFF77EFE236A0133F2D004F1180000F017
:1027D00081F8EDE7F0B5234F234D3E4687B0BD426B
:1027E00005F1300414D3214B9A68D37B013BD3739A
:1027F0004FF02003EFF3118583F311881A4CB44294
:1028000023D385F3118807B0BDE8F040FFF782BEFF
:1028100054F8043C059354F8103C049354F8143CC9
:10282000039354F8183C029354F81C3C019354F859
:10283000203C009354E90A2354E90C01FFF790FF70
:1028400054F8303CDD642546C9E7616A4B1C03D06F
:10285000206819B9FFF76CFF3034D0E7FFF724FF89
:10286000FAE700BF300F0020300F002020010020C9
:1028700003730023C3734FF0FF334273817303620A
:1028800070470000034B1B680BB9FEF73BBC0020F0
:10289000704700BF100100204FF02003EFF31180BC
:1028A00083F3118870470000036840B1084A5268FA
:1028B000904204D01BB19A6881680A449A604268C9
:1028C000136003685A604FF0FF338360704700BFA6
:1028D000B00E002010B50246FFF7DEFF04469068F8
:1028E000431C03D01046FFF7DFFF002084F311885C
:1028F00010BD0000134B70B51B78002B14BF4FF0B8
:10290000FF326FF00042FFF7C7FF0F4B06461C680F
:102910009C420AD04CB1A568FFF7B4FF281A0028E2
:102920000DDBA468FFF7AEFF221A86F31188074B70
:102930001B6913B19A42A8BF1A46104670BD002207
:10294000F3E700BF14010020B00E0020200100209A
:1029500070B5C16016460446FFF79EFF0546FFF7B7
:1029600091FF012EACBF80190130164BA0601A6890
:102970009A4201D05E6832B95A68236062605A6830
:1029800014605C600BE09068A168884214DD411A15
:1029900091605168C4E9002151680C6054601A6864
:1029A0009A4206D0944204D1FFF7A4FF0021FEF71B
:1029B00075FB85F3118870BD091A9642A160DBD0C2
:1029C0001268D8E7B00E00202DE9F04B04464FF016
:1029D0000008204D204E214FFFF728FE2C60FFF706
:1029E0005BFF34688146B4421CD094B1A1682B6867
:1029F000994215DC5B1A2B60D7E9002312EB010B1F
:102A000043EBE17CC4F808802046C7E900BCFFF72F
:102A10004BFF89F311883CB1E36820469847DEE715
:102A2000C91AA1600024F4E7FFF736FF0B490646F8
:102A3000D1E9002328682C60171843EBE078C1E93E
:102A40000078FFF757FF2146FEF728FB86F3118831
:102A5000BDE8F08B10010020B00E0020180100200E
:102A600070B50E460446FFF717FF0546FFF742FF15
:102A7000431C01D0A04203DD31462046FEF70EFB89
:102A800085F3118870BD000038B5074C074DAC4286
:102A900001D3002038BD04F114032046C4E90533F6
:102AA000FDF7B8FE1C34F2E7300F0020300F002095
:022AB00070476D
:022AB200FFFF24
:082AB4005CD7FF7F0100000068
:102ABC0000000000851600000000000085160000D4
:102ACC0000000000851600000000000085160000C4
:102ADC00000000008516000000000000910E0000B0
:102AEC0000000000851600000000000085160000A4
:102AFC000000000085160000000000008516000094
:102B0C000000000085160000000000008516000083
:102B1C00000000008516000000000000891D000068
:102B2C000000000085160000000000008516000063
:102B3C000000000085160000000000008516000053
:102B4C000000000085160000000000008516000043
:102B5C00000000008516000000000000D90F0000E6
:102B6C000000000085160000000000008516000023
:102B7C000000000085160000000000008516000013
:102B8C000000000085160000000000008516000003
:102B9C0000000000851600000000000085160000F3
:102BAC0000000000851600000000000085160000E3
:102BBC0000000000851600000000000085160000D3
:102BCC0000000000851600000000000085160000C3
:102BDC0000000000851600000000000085160000B3
:102BEC0000000000851600000000000085160000A3
:102BFC000000000085160000000000008516000093
:102C0C000000000085160000000000008516000082
:102C1C000000000085160000000000008516000072
:102C2C000000000085160000000000008516000062
:102C3C000000000085160000000000008516000052
:102C4C000000000085160000000000008516000042
:102C5C000000000085160000000000008516000032
:102C6C000000000085160000000000008516000022
:102C7C000000000085160000000000008516000012
:102C8C000000000085160000000000008516000002
:102C9C0000000000851600000000000085160000F2
:102CAC0000000000851600000000000085160000E2
:082CBC00000000008516000075
:102CC4008C300000050C0000000000008C30000077
:102CD400B90D000000000000242F0000FF0E0000CA
:102CE400000000002F2F0000FF0E00000000000075
:102CF4003A2F000019100000000000008C30000082
:102D0400C518000000000000B4340000311C0000AD
:102D1400AC340000BB34000071210000E03400003A
:102D2400032F000051210000D83400008C30000033
:082D3400892A000000000000E4
:102D3C001D0000001C0000001A0000001B00000019
:102D4C00120000001100000015000000130000002C
:102D5C0053656375726520426F6F743A20636F6EB2
:102D6C0066696775726520666C6173680A005365E5
:102D7C006375726520426F6F743A205350553A2038
:102D8C0073657420726567696F6E20257520617399
:102D9C00205365637572650A00536563757265200F
:102DAC00426F6F743A205350553A20736574204625
:102DBC006C61736820726567696F6E202575206180
:102DCC0073204E6F6E2D5365637572650A005365E3
:102DDC006375726520426F6F743A20636F6E66691B
:102DEC0067757265205352414D0A005365637572C5
:102DFC006520426F6F743A205350553A20736574B6
:102E0C00205352414D20726567696F6E20257520E5
:102E1C006173205365637572650A0053656375723F
:102E2C006520426F6F743A205350553A2073657485
:102E3C00205352414D20726567696F6E20257520B5
:102E4C006173204E6F6E2D5365637572650A005366
:102E5C00656375726520426F6F743A20636F6E669E
:102E6C006967757265207065726970686572616CEE
:102E7C00730A0053656375726520426F6F743A2054
:102E8C004D53505F4E532025780A0053656375727D
:102E9C006520426F6F743A207072657061726520A4
:102EAC00746F206A756D7020746F204E6F6E2D5389
:102EBC00656375726520696D6167650A00000000C5
:102ECC0002000000D42E000000000000F42E0000D0
:102EDC0006000000E0FF0F0000000020FC2E0000A8
:102EEC0021000000E0FF0020464C4153485F3000B9
:102EFC005352414D5F3000554152545F3000000039
:102F0C00350E00000000000000000000150F00004E
:102F1C00D50D000000000000636C6B5F6B333273E7
:102F2C00726300636C6B5F6D31367372630073791F
:102F3C00735F636C6F636B002A2A2A2A2A2042551E
:102F4C0053204641554C54202A2A2A2A2A0A00206A
:102F5C0020507265636973652064617461206275C9
:102F6C0073206572726F720A002020424641522013
:102F7C00416464726573733A20307825780A0020B6
:102F8C0020496D707265636973652064617461209A
:102F9C00627573206572726F720A002020496E731D
:102FAC007472756374696F6E2062757320657272CA
:102FBC006F720A005265736572766564204578639A
:102FCC00657074696F6E20280053707572696F7527
:102FDC007320696E74657272757074202849525131
:102FEC00200020205320696E737472756374696FAE
:102FFC006E20616464726573733A20203078257892
:10300C000A00524554544F4241534520646F657336
:10301C00206E6F74206D61746368204558435F5255
:10302C00455455524E0A002A2A2A2A2A204841522F
:10303C0044204641554C54202A2A2A2A2A0A002088
:10304C0020427573206661756C74206F6E207665F6
:10305C0063746F72207461626C6520726561640ABE
:10306C000020204661756C7420657363616C61741B
:10307C00696F6E20287365652062656C6F77290A0D
:10308C00002A2A2A2A2A204465627567206D6F6EF1
:10309C0069746F7220657863657074696F6E20282F
:1030AC006E6F7420696D706C656D656E74656429E6
:1030BC00202A2A2A2A2A0A002A2A2A2A2A2025737E
:1030CC0020256429202A2A2A2A2A0A002A2A2A2A7E
:1030DC002A204D5055204641554C54202A2A2A2A44
:1030EC002A0A002020537461636B696E6720657235
:1030FC00726F720A002020556E737461636B696E77
:10310C0067206572726F720A00202044617461201E
:10311C004163636573732056696F6C6174696F6E7C
:10312C000A0020204D4D4641522041646472657363
:10313C00733A20307825780A002020496E73747217
:10314C00756374696F6E2041636365737320566990
:10315C006F6C6174696F6E0A002020466C6F61742D
:10316C00696E672D706F696E74206C617A7920734B
:10317C007461746520707265736572766174696FC1
:10318C006E206572726F720A002A2A2A2A2A20532C
:10319C004543555245204641554C54202A2A2A2A4B
:1031AC002A0A002020416464726573733A203078D7
:1031BC0025780A002020496E76616C696420656E62
:1031CC0074727920706F696E740A002020496E76D3
:1031DC00616C696420696E746567726974792073B7
:1031EC0069676E61747572650A002020496E76619C
:1031FC006C696420657863657074696F6E207265A4
:10320C007475726E0A002020417474726962757450
:10321C00696F6E20756E69742076696F6C61746964
:10322C006F6E0A002020496E76616C69642074729E
:10323C00616E736974696F6E0A0020204C617A7933
:10324C002073746174652070726573657276617435
:10325C00696F6E0A0020204C617A79207374617456
:10326C0065206572726F720A002A2A2A2A2A205552
:10327C0053414745204641554C54202A2A2A2A2A94
:10328C000A0020204469766973696F6E2062792088
:10329C007A65726F0A002020556E616C69676E65E5
:1032AC0064206D656D6F7279206163636573730A59
:1032BC00002020537461636B206F766572666C6FAF
:1032CC00770A0020204E6F20636F70726F636573F6
:1032DC00736F7220696E737472756374696F6E7339
:1032EC000A002020496C6C6567616C206C6F61640E
:1032FC00206F66204558435F52455455524E206905
:10330C006E746F2050430A002020496C6C65676115
:10331C006C20757365206F6620746865204550536A
:10332C00520A002020417474656D707420746F20F3
:10333C006578656375746520756E646566696E6520
:10334C006420696E737472756374696F6E0A002AF7
:10335C002A2A2A2A2048617264776172652065786E
:10336C0063657074696F6E202A2A2A2A2A0A002A39
:10337C002A2A2A204B65726E656C20416C6C6F6337
:10338C006174696F6E204661696C75726521202AC3
:10339C002A2A2A0A002A2A2A2A2A204B65726E65B2
:1033AC006C204F4F505321202A2A2A2A2A0A002AFD
:1033BC002A2A2A2A204B65726E656C2050616E6930
:1033CC006321202A2A2A2A2A0A002A2A2A2A205554
:1033DC006E6B6E6F776E20466174616C20457272F5
:1033EC006F7220256421202A2A2A2A0A004375722A
:1033FC0072656E7420746872656164204944203D66
:10340C002025700A4661756C74696E6720696E734D
:10341C007472756374696F6E206164647265737322
:10342C00203D20307825780A00495352006573738B
:10343C00656E7469616C20746872656164004661C4
:10344C0074616C206661756C7420696E2025732123
:10345C00205370696E6E696E672E2E2E0A004661BF
:10346C0074616C206661756C7420696E207468726E
:10347C00656164202570212041626F7274696E67EA
:10348C002E0A0000611C0000451B0000791B000087
:10349C00AB1B0000AD1E0000ED1B00000000000087
:1034AC0000258450000000004750494F5F30005504
:1034BC004152545F320000005D200000812000006A
:1034CC00AF200000ED1E00004D20000000800050D9
:1034DC000100000000A0005001000000B80E002008
:1034EC00180F0020240F0020300F0020300F002078
:1034FC00F5FFFFFF6D61696E0069646C650000008B
:10350C00300000202A2A2A2A2A20426F6F74696E02
:10351C0067205A6570687972204F532076312E31AE
:10352C00332E39392D6E637332202A2A2A2A2A0A1D
:04353C00000000008B
:10354000AB0800000090D0038025000000010300BC
:1035500000000000004B000000010300000000001C
:08356000B00E0020B00E0020A7
:10356800C42C00000000000000000000302D000006
:103578000000000000000000002D00000000000016
:1035880000000000DC2C00000C2F000000000000F0
:10359800E82C0000182F000000000000182D000083
:1035A800C4340000A40E0020242D0000C434000000
:1035B800980E0020D02C0000000000000000000041
:1035C800F42C000000000000000000000C2D00009A
:0835D8009034000010000020F7
:1035E000300F0020300F002000000000000000001D
:0435F0000F000000C8
:0400000300001839A8
:00000001FF
